:100000000C949E000C94C6000C94C6000C94C60080
:100010000C94C6000C94C6000C94D4060C94C60034
:100020000C94C6000C94C6000C94C6000C94C60038
:100030000C94C6000C94C6000C94C6000C94C60028
:100040000C94D0090C94C6000C9406090C94380941
:100050000C94C6000C94C6000C94C6000C94C60008
:100060000C94C6000C94C6000C94C6000C94C600F8
:100070000C94C6000C94C6000C94C6000C94C600E8
:100080000C94C6000C94C6000C94C6000C94EA00B4
:100090000C94C6000C94C6000C94C6000C94C600C8
:1000A0000C94C6000C94C6000C94C6000C94C600B8
:1000B0000C94C600FF060207F506F906230723077E
:1000C00006070A071007140723071A071E07090C5B
:1000D0000D080002010000030407000000000000FA
:1000E000000000000000010204081020408001020E
:1000F000040810200102040810200102040804046E
:1001000004040404040402020202020203030303BF
:100110000303050505050000000023002600290053
:100120002C0000000000250028002B002E000000FD
:100130000000240027002A002D00680911241FBE9A
:10014000CFEFD8E0DEBFCDBF11E0A0E0B1E0E0E648
:10015000F5E102C005900D92AC39B107D9F722E064
:10016000ACE9B1E001C01D92A639B207E1F710E099
:10017000CEE9D0E004C02197FE010E948E0ACD395D
:10018000D107C9F70E9496090C94AE0A0C9400009E
:1001900084E680939C0161E082E00E946007A8955C
:1001A00080919C018111F7CF60E082E00C946007A0
:1001B00010929000E1E9F0E0108285E89FEF9093C3
:1001C00095008093940081E08093710088BB82E069
:1001D000808308951F920F920FB60F9211242F93D0
:1001E0003F934F935F936F937F938F939F93AF93BF
:1001F000BF93EF93FF9385E89FEF909395008093D3
:1002000094008091AD01882319F081508093AD0155
:1002100084E00E9490079091A401813099F410929B
:10022000A701913009F19091A6019F5F923318F4D4
:100230009093A60119C01092A6018093A401109278
:10024000AA0112C01092A601992371F08091A70112
:100250008F5F823318F48093A70106C01092A70124
:100260001092A4011092AA0180919F018F5F8436A1
:1002700018F480939F013DC010929F0180919C01D2
:10028000882319F0815080939C0180919E018F5F9B
:100290008A3018F480939E012CC010929E018091A8
:1002A000AA01882319F081508093AA0180919D01B1
:1002B0008F5F8C3318F480939D011BC010929D01B9
:1002C0008091A0019091A101009729F0019790934E
:1002D000A1018093A0018091A201882319F081508F
:1002E0008093A2018091A301882319F0815080930B
:1002F000A301FF91EF91BF91AF919F918F917F915A
:100300006F915F914F913F912F910F900FBE0F9082
:100310001F901895E0EAF1E080EA95E091838083F0
:100320008AE0828383830895E0EAF1E082E08483B7
:10033000168217828CE381878287108615820C943F
:100340008A01EBEAF1E01082118212821382148298
:1003500008950FB6F894A895809160008861809305
:100360006000109260000FBE61E082E00E942407EE
:1003700062E084E00E94240762E081E10E94240799
:1003800060E082E00E94600726E040E855E260E01D
:1003900070E080EF91E00E94A6080E94D800789457
:1003A0009FE088E10FB6F894A895809360000FBE97
:1003B000909360000E9494010C94A10190E0981722
:1003C00079F0421768F4FB01E40FF11D30813C32F3
:1003D00011F49F5F03C03A3209F4982F4F5FEFCFBB
:1003E000842F08958053873130F4E82FF0E0E05FE8
:1003F000FE4F808108958FEF0895BF92CF92DF92D4
:10040000EF92FF920F931F93CF93DF93B82E8A0141
:10041000C62F6B3008F0CAE0C150D0E0C12CD12CFF
:1004200076018C2F8B0DF801E80FF11D80810E9461
:10043000F2018A3098F494E0D99FF0011124E95A2E
:10044000FE4F2081318142815381A82FB0E00E946C
:10045000940AC60ED71EE81EF91EDF5FC15008F7CA
:10046000C701B601DF91CF911F910F91FF90EF90DF
:10047000DF90CF90BF900895CF92DF92EF92FF92DE
:100480000F931F93CF93DF93D82F7B01D42EC22ECF
:100490000E94DE01C82F2C2D4D2DB70181E08D0F5C
:1004A0000E94DE01482F50E02C2F30E02F5F3F4F9D
:1004B0004217530779F09FEF980F692F6C1BA70124
:1004C0008C2F0E94FD01F8016083718382839383E6
:1004D00081E001C080E0DF91CF911F910F91FF90EB
:1004E000EF90DF90CF9008959F92AF92BF92CF92FE
:1004F000DF92EF92FF920F931F93CF93DF93C62F5C
:10050000590199249394D0E0C12CD12C76018A0111
:10051000080F191FF801EC0FF11D319780810E941F
:10052000F2018031A0F494E0D99FF0011124E95C3C
:10053000FE4F2081318142815381A82FB0E00E947B
:10054000940AC60ED71EE81EF91EDF5F01C0912C6B
:10055000C15001F7F5019082C701B601DF91CF913B
:100560001F910F91FF90EF90DF90CF90BF90AF90D1
:100570009F9008959F92AF92BF92CF92DF92EF9299
:10058000FF920F931F93CF93DF931F92CDB7DEB7E8
:10059000B82E6B01A42E922E1982882329F00E9476
:1005A000DE01E82EF12C02C0E12CF12C292D4A2D80
:1005B000B60181E08B0D0E94DE01482F50E09701CB
:1005C0002F5F3F4F2417350789F08150682F6E1930
:1005D0009E012F5F3F4FA601C7010E947402F801E0
:1005E000608371838283938381E001C080E00F90F8
:1005F000DF91CF911F910F91FF90EF90DF90CF90FF
:10060000BF90AF909F900895CF93DF9390E0FA0151
:10061000E90FF11D3081332311F09F5FF8CF2917C7
:1006200019F0222311F017C020E031E0A82FB0E02C
:10063000291790F4E22FF0E0EB01CE0FDF1FCA0F75
:10064000DB1FE40FF51FC8818081C81711F0292F27
:1006500030E02F5FEDCF30E0832FDF91CF91089511
:10066000EF92FF921F93CF93DF93DC01F901108289
:100670006F5F7D01E60EF11CE70198819A3239F037
:100680006417B8F48081982790836F5FF2CF641766
:1006900080F4EF01F70181810E94F201182F129579
:1006A000107FF70182810E94F201180F81E098818A
:1006B000191380E0DF91CF911F91FF90EF90089583
:1006C0009091AC01E92FF0E0E555FE4F85A3903203
:1006D00018F49F5F9093AC019091AE01913029F492
:1006E0009091AF0189278093AF0108950F931F93D5
:1006F000CF938C01C0E0F801EC0FF11D80818823BD
:1007000021F00E946003CF5FF6CFCF911F910F9130
:1007100008958F929F92AF92BF92CF92DF92EF9205
:10072000FF921F93CF93DF936B017C01C42FD22FD5
:10073000411103C010E0CAE001C011E0C15084E0E3
:10074000C89FF0011124E95AFE4F80809180A28059
:10075000B380C701B601A50194010E946C0A113053
:1007600039F4F901E95DFE4F80810E94600315C0F4
:10077000211531054105510541F0F901E95DFE4FB3
:1007800080810E94600311E008C0C11105C080E3B0
:100790000E94600310E001C010E0C701B601A5018E
:1007A00094010E946C0A6B017C01C111C7CFD1304A
:1007B00029F48DE00E9460038AE003C0DD2371F01C
:1007C0008D2FDF91CF911F91FF90EF90DF90CF9011
:1007D000BF90AF909F908F900C946003DF91CF916A
:1007E0001F91FF90EF90DF90CF90BF90AF909F90C0
:1007F0008F9008958F929F92AF92BF92CF92DF9287
:10080000EF92FF921F93CF93DF936B017C01C42F74
:10081000D22F411103C010E0C9E001C011E0C15066
:1008200084E0C89FF0011124E95CFE4F8080918034
:10083000A280B380C701B601A50194010E946C0A91
:10084000113039F4F901E95DFE4F80810E946003A7
:1008500015C0211531054105510541F0F901E95D4A
:10086000FE4F80810E94600311E008C0C11105C0E5
:1008700080E30E94600310E001C010E0C701B601F0
:10088000A50194010E946C0A6B017C01C111C7CFC4
:10089000D13029F48DE00E9460038AE003C0DD239B
:1008A00071F08D2FDF91CF911F91FF90EF90DF902E
:1008B000CF90BF90AF909F908F900C946003DF918A
:1008C000CF911F91FF90EF90DF90CF90BF90AF90AE
:1008D0009F908F900895CF93C0E08091AC01C8178E
:1008E00058F4EC2FF0E0E555FE4F65A180EF91E064
:1008F0000E945908CF5FF1CF80EF91E0CF910C9427
:1009000037080F931F93CF93DF930BEA11E0F801A1
:10091000118284E20E946003F801148281E08383E3
:1009200080E091E00E9476032CE241E061E070E01B
:1009300080E090E00E948903C0EAD1E06C8170E021
:1009400080E090E02CE241E00E948903688570E03D
:1009500080E090E02CE241E00E9489036A8170E02F
:1009600080E090E02CE240E00E9489036881798178
:1009700080E090E02CE240E00E948903698570E00D
:1009800080E090E02CE240E00E94890386E891E05C
:100990000E9476038CE20E9460036B8170E080E02D
:1009A00090E020E040E00E948903F80113828AE28F
:1009B0000E946003F801648170E080E090E021E033
:1009C00042E00E94FA03DF91CF911F910F910C94A6
:1009D0006B04CF93DF93CBEAD1E0198284E20E94CB
:1009E00060031C8281E08B8380E091E00E947603AB
:1009F0002CE241E064E070E080E090E00E94890336
:100A000020E043E06DE770E080E090E00E94890321
:100A10001B828AE20E9460036C8170E080E090E0BB
:100A200021E042E00E94FA03DF91CF910C946B0425
:100A3000CF93DF93CBEAD1E0198284E20E94600376
:100A40001C8281E08B8385E091E00E9476031B820B
:100A50008AE20E9460036C8170E080E090E021E017
:100A600042E00E94FA03DF91CF910C946B04EF9265
:100A7000FF920F931F93CF93DF9300D000D000D04D
:100A8000CDB7DEB719821A821B821C821D829E019D
:100A90002B5F3F4F4091AB0160E080EB91E00E9403
:100AA0003003813009F0F5C020E04FE751E060EB02
:100AB00071E080E00E940403813009F0EAC08E01F9
:100AC0000F5F1F4F2091AB0140E060EB71E00E948F
:100AD0003C02813011F4898101C080E01092A501AF
:100AE000833009F458C018F4813041F0D2C084300A
:100AF00009F498C0803509F4B2C0CBC08E010F5FF5
:100B00001F4F2091AB0140E060EB71E082E00E945A
:100B10003C02813011F4F98001C0F12C8E010F5F8D
:100B20001F4F2091AB0140E060EB71E083E00E9439
:100B30003C02813011F4E98001C0E12C2091AB012D
:100B400030E08E010F5F1F4F40E050E060EB71E03E
:100B500084E00E94BA02813019F4898187FF04C0C1
:100B60008AE08093A30104C084FDFACF8076C1F3AC
:100B70008FEF8F0D863018F481E0E81206C080EA0E
:100B800095E09093A1018093A0018AE08093A20157
:100B90000E9481047EC08E010F5F1F4F2091AB0128
:100BA00040E060EB71E082E00E943C02813011F491
:100BB000998101C090E08E010F5F1F4F2091AB0122
:100BC00040E060EB71E083E09E830E943C029E81E6
:100BD000813021F5923019F0903869F01DC089817B
:100BE0009A81AB81BC8182309105A105B105A0F449
:100BF0008093A80111C089819A81AB81BC81AC012D
:100C0000BD0141505109610971094C33510561051C
:100C1000710510F48093A9010E9481048AE08093F9
:100C2000A20137C08E010F5F1F4F2091AB0140E042
:100C300060EB71E082E00E943C02813079F74981EB
:100C40005A816B817C81413051056105710531F715
:100C50008E830E94E9048E818093A501DFCF8E01EF
:100C60000F5F1F4F2091AB0140E060EB71E082E02D
:100C70000E943C02813069F489819A81AB81BC81F8
:100C80008D379105A105B10521F40E9418050E9438
:100C90008A0126960FB6F894DEBF0FBECDBFDF9156
:100CA000CF911F910F91FF90EF9008951F93CF93D5
:100CB000DF9380EF91E00E94B907892BA9F1109290
:100CC000AB0112E3A89580EF91E00E94B907892B50
:100CD00011F180EF91E00E94B907C091AB01D0E023
:100CE000892B79F080EF91E00E94D307C555DE4F44
:100CF0008D838091AB01803260F78F5F8093AB0171
:100D0000E8CFC555DE4F8C818A3019F41092AD01C1
:100D100002C01093AD018091AD018111D3CFDF915D
:100D2000CF911F910C943705DF91CF911F910895BA
:100D30007894A89561E082E00E94240760E082E058
:100D40000E94600762E084E00E94240762E081E183
:100D50000E9424070E9456068091A501813039F433
:100D60000E948A018091A9018093AA01E1CF80911C
:100D7000AA01811106C00E9481048091A90180937B
:100D8000AA018091A0019091A101892B41F080914D
:100D9000A201882321F08091A3018111C9CF0E9473
:100DA000C8000E948A01C4CF1F920F920FB60F9203
:100DB00011248F930FB6F894A895809160008861F4
:100DC00080936000109260000FBE8F910F900FBE55
:100DD0000F901F90189590E0FC013197ED30F105D0
:100DE00090F5E65AFF4F0C948E0A809180008F7721
:100DF00003C0809180008F7D80938000089584B52A
:100E00008F7702C084B58F7D84BD08958091B00036
:100E10008F7703C08091B0008F7D8093B0000895DC
:100E2000809190008F7703C0809190008F7D809398
:100E3000900008958091A0008F7703C08091A0005A
:100E40008F7D8093A0000895CF93DF9390E0FC0105
:100E5000EA51FF4F2491FC01E250FF4F8491882317
:100E600061F190E0880F991FFC01E25DFE4FC59192
:100E7000D491FC01EE5DFE4FA591B491611109C0C2
:100E80009FB7F8948881209582238883EC912E2344
:100E90000BC0623061F49FB7F8943881822F80953F
:100EA00083238883EC912E2B2C939FBF06C08FB792
:100EB000F894E8812E2B28838FBFDF91CF9108957E
:100EC0001F93CF93DF93282F30E0F901E253FF4FB8
:100ED0008491F901EA51FF4FD491F901E250FF4F9B
:100EE000C491CC23C9F0162F81110E94EB06EC2F80
:100EF000F0E0EE0FFF1FEE5DFE4FA591B4918FB7AE
:100F0000F894111105C09C91ED2FE095E92302C0E2
:100F1000EC91ED2BEC938FBFDF91CF911F91089552
:100F2000CF93DF93282F30E0F901E253FF4F8491F4
:100F3000F901EA51FF4FD491F901E250FF4FC491FA
:100F4000CC2391F081110E94EB06EC2FF0E0EE0F24
:100F5000FF1FEA5EFE4FA591B491EC91ED2381E075
:100F600090E021F480E002C080E090E0DF91CF913A
:100F70000895FC01918D228D892F90E0805C9F4F18
:100F8000821B91098F7399270895FC01918D828DA1
:100F9000981731F0828DE80FF11D858D90E008954E
:100FA0008FEF9FEF0895FC01918D828D981761F06E
:100FB000828DDF01A80FB11D5D968C91928D9F5F90
:100FC0009F73928F90E008958FEF9FEF0895FC013B
:100FD000538D448D252F30E0842F90E0821B930B9E
:100FE000541710F0CF960895019708958EE599E073
:100FF000892B41F080E090E0892B21F00E945E096E
:1010000081110DC080E090E0892B71F080E090E0CC
:10101000892B51F00E940000811104C008950E94A4
:101020000000F0CF0C9400000895FC01848DDF01D6
:10103000A80FB11DA35ABF4F2C91848D90E001964B
:101040008F739927848FA689B7892C93A089B1893A
:101050008C91837080648C93938D848D981306C0DB
:101060000288F389E02D80818F7D80830895CF935E
:10107000DF93EC01888D8823C9F0EA89FB898081A0
:1010800085FD05C0A889B9898C9186FD0FC00FB672
:1010900007FCF5CF808185FFF2CFA889B9898C91B3
:1010A00085FFEDCFCE010E941508E7CFDF91CF91EC
:1010B0000895EF92FF920F931F93CF93DF93EC016C
:1010C00081E0888F9B8D8C8D981305C0E889F98904
:1010D000808185FD26C0F62E0B8D10E00F5F1F4F1F
:1010E0000F731127E02E8C8DE8120CC00FB607FC91
:1010F000FACFE889F989808185FFF5CFCE010E947A
:101100001508F1CF8B8DFE01E80FF11DE35AFF4F5B
:10111000F0829FB7F8940B8FEA89FB898081806207
:101120000AC09FB7F894EE89FF896083E889F9893E
:1011300080818370806480839FBF81E090E0DF9135
:10114000CF911F910F91FF90EF900895CF92DF9272
:10115000EF92FF921F93CF93DF93EC016A017B0123
:10116000122F60E970ED83E090E0A70196010E94E4
:101170006C0ADA01C9010197A109B109B695A795D1
:1011800097958795AC01E889F98982E080834115BC
:1011900080E15807A8F0E889F989108268E478EEC0
:1011A00081E090E0A70196010E946C0ABA01A901B2
:1011B0004150510961097109769567955795479591
:1011C000EC85FD855083EE85FF854083188EEC8984
:1011D000FD891083EA89FB89808180618083EA89A7
:1011E000FB89808188608083EA89FB8980818068AF
:1011F0008083EA89FB8980818F7D8083DF91CF9115
:101200001F91FF90EF90DF90CF9008951F920F9263
:101210000FB60F9211242F938F939F93EF93FF9309
:10122000E0910002F09101028081E0910602F091CC
:10123000070282FD12C09081809109028F5F8F7337
:1012400020910A02821751F0E0910902F0E0E0518A
:10125000FE4F958F8093090201C08081FF91EF912D
:101260009F918F912F910F900FBE0F901F90189507
:101270001F920F920FB60F9211242F933F934F930B
:101280005F936F937F938F939F93AF93BF93EF93EE
:10129000FF9380EF91E00E941508FF91EF91BF91BD
:1012A000AF919F918F917F916F915F914F913F91FE
:1012B0002F910F900FBE0F901F90189580EF91E027
:1012C0000E94B90721E0892B09F420E0822F0895BC
:1012D000E0EFF1E01382128288EE93E0A0E0B0E04C
:1012E00084839583A683B7838EE891E0918380837E
:1012F00085EC90E09587848784EC90E097878687DB
:1013000080EC90E0918B808B81EC90E0938B828BD2
:1013100082EC90E0958B848B86EC90E0978B868BAB
:10132000118E128E138E148E089508950E941A0A3B
:101330000E9495090E94A901C6EFD7E00E94980675
:101340002097E1F30E94F607F9CFCF92DF92EF9258
:10135000FF920F931F93CF93DF936C017A018B0160
:10136000C0E0D0E0CE15DF0589F0D8016D918D0188
:10137000D601ED91FC910190F081E02DC601099517
:10138000892B11F47E0102C02196ECCFC701DF91B9
:10139000CF911F910F91FF90EF90DF90CF90089524
:1013A0001F920F920FB60F9211242F933F938F939A
:1013B0009F93AF93BF9380918E0290918F02A091E3
:1013C0009002B091910230918D0220E3230F2D37CE
:1013D00020F44096A11DB11D05C023EB230F4196BB
:1013E000A11DB11D20938D0280938E0290938F02D8
:1013F000A0939002B09391028091920290919302F7
:10140000A0919402B09195020196A11DB11D809307
:10141000920290939302A0939402B0939502BF918D
:10142000AF919F918F913F912F910F900FBE0F9091
:101430001F901895789484B5826084BD84B58160CE
:1014400084BD85B5826085BD85B5816085BDEEE6CC
:10145000F0E0808181608083E1E8F0E010828081AB
:1014600082608083E0E8F0E0808181608083E1EB4E
:10147000F0E0808184608083E0EBF0E08081816037
:101480008083E1E9F0E080818260808380818160F7
:101490008083E0E9F0E0808181608083E1EAF0E030
:1014A000808182608083808181608083E0EAF0E0D7
:1014B000808181608083EAE7F0E080818B7F808398
:1014C0008081826080838081816080838081806868
:1014D00080831092C1000895A1E21A2EAA1BBB1BA3
:1014E000FD010DC0AA1FBB1FEE1FFF1FA217B307F0
:1014F000E407F50720F0A21BB30BE40BF50B661F06
:10150000771F881F991F1A9469F7609570958095C9
:1015100090959B01AC01BD01CF010895EE0FFF1F17
:101520000590F491E02D09940E949F0AA59F900DCB
:10153000B49F900DA49F800D911D11240895A29F2A
:10154000B001B39FC001A39F700D811D1124911D97
:10155000B29F700D811D1124911D0895F894FFCF45
:101560005649472C005649472C38302C313235002B
:1015700000010203040506070809FFFFFFFFFFFF44
:10158000FF0A0B0C0D0E0F3031323334353637383D
:10159000394142434445460100000010000000006C
:1015A0000100000010000000000100000010000019
:1015B00000000100000010010000000A00000064AB
:1015C000000000E803000010270000A08601004092
:1015D000420F008096980000E1F50500CA9A3B246E
:1015E0004D4632302C00312E3200000000005908E8
:0C15F000A509E7073708B907D307C507AE
:00000001FF
